:020000020000FC
:1000000019C05BC15BC1FCCFFCCFFCCFA0C19EC1BE
:100010009CC156C156C156C156C156C195C193C166
:1000200054C15BC15BC15BC15BC15BC187C187C19F
:1000300088C188C102E00EBF0FEF0DBF0FEF0AB9F4
:1000400004B905B900270BB90027009300010093FC
:100050000101009302010093030100930401009346
:100060000501009306010093070101E000937C0065
:100070000EE800937A0003E005BD01E000936E00F6
:10008000F894002706BD7894DAD033D0FCCFF894EA
:1000900000270093070100930301009304010093DC
:1000A00005010093060101E000937C007894089517
:1000B000F89401E0009307010027009303010093E7
:1000C0000401009305010093060103E000937C0006
:1000D0007894089500910701003011F0D8DF08C02E
:1000E0000BE000930001009301010AE0009302017C
:1000F00008950091060111E0011308950091040193
:100100001091050126E0169507952A95E1F722271B
:1001100020930401209305012093060120930301FD
:100120000456120BEAF00456120B2AF10456120B75
:1001300032F10456120B3AF10456120B42F10456F6
:10014000120B4AF10456120B52F10456120B5AF1DB
:100150000456120B62F10456120B6AF1BBDF6EC03B
:100160003091070120E0231302C0A2DF67C030E016
:100170003093020123C031E0309302011FC032E00E
:10018000309302011BC033E03093020117C034E00A
:100190003093020113C035E0309302010FC036E006
:1001A000309302010BC037E03093020107C038E002
:1001B0003093020103C039E0309302010C590A5018
:1001C0009AF00A50AAF00A50BAF00A50CAF00A503F
:1001D000DAF00A50EAF00A50FAF00A500AF10A502E
:1001E0001AF10A502AF12AC030E03093010123C0ED
:1001F00031E0309301011FC032E0309301011BC098
:1002000033E03093010117C034E03093010113C093
:1002100035E0309301010FC036E0309301010BC08F
:1002200037E03093010107C038E03093010103C08B
:1002300039E030930101065F0093000108951091A9
:1002400000010FED009505B91DD01BB92BD0109101
:1002500001010FEE009505B915D01BB900910701FA
:10026000003009F45B981ED0109102010FE7009551
:1002700005B908D01BB900910701013009F45B985A
:1002800011D00895E6E9F2E020E0E10FF21FC895F1
:10029000102D10950895F505735787D6F645F7D7B5
:1002A000F22200021F932F931EE12EE11A95F1F71F
:1002B0002A95E1F72F911F91089518951895189593
:1002C000189518951895189518950F93F89403E0BC
:1002D00003BF78940F9188951895189518951895DF
:1002E00018950F931F932F933F939FB7009106018B
:1002F0000130F1F0009103010034A1F000910301FD
:1003000003950093030110917800009179002091EA
:10031000050130910401310F201F30930401209317
:10032000050106C000270093030101E000930601C8
:100330009FBF3F912F911F910F9118951895189578
:100340001895189518951895189518951895189545
:00000001FF
